:0600000000008A011C282B
:08000800090050347234653424
:1000100073347334203445345334433420347434CB
:100020006F34203465346E346434003444346F34B7
:100030006E34653421340034833083160313810019
:1000400083128B120B17313090006030F80097202C
:1000500029280530F0000030F100AD200D30A1203E
:100060000A30A120831603130613831206138C1E75
:100070003E280130F0000030F1004028F001F1018D
:10008000F201F301B82003194A28BF208312031399
:10009000A0004B2837282008F000F1011B30F200A7
:1000A0000030F300B82003195828F001F1015C2852
:1000B0000130F0000030F100F201F301B820031923
:1000C00062288828831203132008F000F1017008C9
:1000D000A120831203132008F000F1010D30F2007B
:1000E0000030F300B82003197828F001F1017C28D2
:1000F0000130F0000030F100F201F301B8200319E3
:1001000087280B30F0000030F1007008A12037285C
:100110000D30A1200A30A1201630F0000030F1008F
:10012000AD200D30A1200A30A12063009528673052
:10013000831603139900181598168312181698172A
:100140000800831203130C1EA32899000800700FE7
:10015000F103F10AF00071040800B420003803191B
:100160000800A120A720AD2871088A00700882002D
:1001700073087102031D08007208700208008312E0
:0A01800003138C1EC1281A080800A2
:00000001FF
